:100000000C948F00189518951895189518951895B3
:100010001895189518951895189518951895189578
:100020001895189518951895189518951895189568
:100030001895189518951895189518951895189558
:100040001895189518951895189518951895189548
:10005000189518953B2F4A2FCA500FEF07BB50C079
:1000600020E0C8992395EC2FA0E6B0E00D91E00FB9
:10007000F0E020830FE916E821E001501040204015
:10008000E1F700C00000E0E6F0E0008111810F5FC1
:100090001F4F00831183A0E6B0E0ED91FC913A97E9
:1000A000FCF21A812B8102E0209F202D210F1C8160
:1000B00004E0109F102D120F2D8108E0209F202DAD
:1000C000210F1E8100E1109F102D120F2F8100E2E1
:1000D000209F202D210F188500E4109F102D120F56
:1000E000298500E8209F010E08BA0FE716E928E9E4
:1000F000015010402040E1F700C0000000E008BBC4
:10010000C89B07C000E010E0E0E6F0E00083118348
:10011000C2CF00E008BBF4CF00008895FECF01EA13
:100120000DBF00E00EBFC2E8D0E00E94A100002396
:1001300011F00E94B1000E942A000E948C000C94D1
:100140008C0001E0089520E006D0E9F7089525919C
:1001500002D0E9F708952D9301501040202F212B54
:10016000089586E991E0FC0105911491FC01329615
:10017000A591B491FC01349625913491422F432BE3
:1001800019F0F901E4DF01C0DEDF069611E08C39D9
:0C019000910748F3089502006000000091
:00000001FF
:00000001FF
